:020000020000FC
:10000000BFC35DC018951895099459C036C018959E
:100010003EC01895189573C01895189518951895A1
:1000200018956DC01895697A40744042405B9FB640
:100030008A9409F4E1E29FBE18959FB68A949FBE08
:10004000189520FD959A21FD979A22FDC09AEDE220
:10005000832C24BC1895A89518958F12EECFA895DF
:1000600011FDEFCFE0916500852C20FD959821FDD5
:10007000979822FDC09844BC18959FB640916300A4
:10008000415008F40E7F409363009FBE18959FB6C1
:10009000409164004395409364004F7019F4BB2075
:1000A00019F0BA949FBE189540916600439540930D
:1000B000660040916700439540936700F3CF4CB5CD
:1000C0005DB5829B0DC09FB65A5659BD48BD42E0F2
:1000D00045BF48E048BF9FBE18959FB6BB240BC0E4
:1000E00098B693FCFACF9FB63A0148B559B5565920
:1000F000641A750A106143E045BF9FBE189590E5EC
:1001000078ECAD98959A17D0E1F7089594E674EBE2
:10011000AB98979A10D0E1F7089598E770EA949811
:10012000C09A09D0E1F708959CE87CE8AB98959ACD
:1001300002D0E1F70895F2BF82B78032E8F39598D4
:100140009798C098949AAD9AAB9A60E1F2BFA8953F
:1001500082B78717E8F36A95C9F79A95089500D092
:1001600000D000D09FE060E1F2BF81E088BFA89599
:1001700088B780FFFDCF6A95B9F79A95A1F70895E2
:10018000809181009091820089569A4739F0C1E8A8
:10019000D0E0E6E285918993C938E1F7089580912E
:1001A000600081BF0F7DC1E8D0E080E890E0A895B5
:1001B000E199FDCF67B760FDFACFC93881F09FBBE9
:1001C0008EBB0196E09A6DB317F06993F0CF7991E9
:1001D0007DBBF894E29A6713E19A7894E8CFC2DF86
:1001E0008FEF81BF0895000C111CAA1C8A95D9F7C6
:1001F0000895869FA12C969FA00CC11DDF1F879F8D
:10020000A00CC11DDF1F979FC00DD11D08951F7643
:10021000C30184369F0708F40895C0917B00D091F4
:100220007C008C1B9D0B60F41068909581959F4F0E
:100230006091790070917A0007C0CC27DD2710C04B
:10024000609177007091780080589140B2F3C8E3D4
:10025000D0E0CFDFC73583E0D80710F0C7E5D3E0A3
:10026000C0937500D093760001FF03C082E0B82EE2
:1002700090C080E1B816BF1E0895809187009091CC
:10028000880080937B0090937C0060918300709144
:100290008400681B790B14D08093770090937800CA
:1002A0006091870070918800809185009091860010
:1002B000681B790B05D08093790090937A0008959C
:1002C0006058714085E595E00196A8959F3F8907A4
:1002D00021F0C0EEDCEF8DDFB9F70895F8948CB50E
:1002E0009DB56091640078B77894903872FD6F1F67
:1002F000C0916800D0916900A0906A008093680066
:100300009093690060936A0000906B0010906C00FD
:1003100070916D00C0936B00D0936C00A0926D0043
:1003200080199109670B97306F0728F480E097E0F8
:1003300060E0D694C7946130A7E5B3E058F062302E
:10034000ACEAB1E038F0643018F080E090E064E0AE
:10035000A6EDD0E07D0180936E0090936F006093D6
:100360007000669597958795C0916800D091690057
:10037000A0906A0073E335D0C0937100D0937200EF
:10038000A092730049D014FD42CFC0917500D09166
:100390007600CE15DF0508F0E701CC15DD0508F085
:1003A000E60187E593E08C1B9D0BB1F02096B1F040
:1003B0001D7F116016FF04C0880F991FCC0FDD1F31
:1003C00071E29F1377E1C09580951E01F8942C018E
:1003D00070936500789408951360F2CF1C7F7DE2DE
:1003E000F2CF879FC10DDF1FAF1E979FC00DD11D9C
:1003F000AF1E679FD00DA11C089580916E00909153
:100400006F0060917000C0917100D0917200A09057
:1004100073000895F2DFE5DF79B7072E7B7E79BFA1
:1004200070E1F894DBBDCABD78BF8CB59DB57894FA
:1004300001606091640078B7903872FD6F1FC81B2F
:10044000D90BA60AA09263000AF40E7F09BE089594
:10045000279670E1F8948CB59DB5C80FD91FDBBD08
:10046000CABD78BFA092630001607894089514FD1E
:10047000CEDE00FDFCCF0895F5BD80E488BFEBE241
:10048000949AAD9AAB9A95989798C0980895829B44
:10049000F09366008091660085FF0895E0E0F8948F
:1004A000FCE185919491F0E0789401960297A8F38D
:1004B000F894F7BBF4BBF1BB88E181BDF1BD80913D
:1004C000600081BF9DCBD9DE84E588BF89BF83E012
:1004D00085BF80E48BBFBB24137EF0936600F0934E
:1004E0006700A89514FD0AC0D2DF809167008837A5
:1004F000C1F78CE38093670010DEF3CF88DEC091F4
:100500007500D0917600209631F78AE0B81648F34E
:10051000812F8C7009F0FBBF07DE06DE05DEACDF45
:100520000D7FF0936600F0936700A89514FD0CC052
:10053000BB20D9F7ACDF809167008E31B1F79CDF2B
:1005400011DEEBDDE3DDBFCF62DE209651F3BB2091
:1005500041F392DF80B7886080BF3798CEE8D0E063
:100560006E010260AAD0F093740082E0B82E86E09B
:10057000809362008CE08093610081E085BD17FD6F
:1005800037C09FD087E087B9AD9A10FD949897D077
:1005900080E087B9F894287F226088B3C09898B328
:1005A0008913979A78948DD086E087B9949A10FD34
:1005B000AB9885D087E087B9F894287F216082B313
:1005C000979892B38913959A78947BD080E087B9F5
:1005D000AB9A10FDAD9873D086E087B9F894287F68
:1005E000246082B3959892B38913C09A789436C0E8
:1005F00066D080E087B9F894287F216088B3C098DE
:1006000098B38913959A78945CD087E087B9AD9AAE
:1006100010FDAB9854D086E087B9F894287F22600B
:1006200082B3959892B38913979A78944AD080E0D0
:1006300087B9AB9A10FD949842D087E087B9F894B7
:10064000287F246082B3979892B38913C09A7894D4
:1006500038D086E087B9949A10FDAD9880916100FA
:10066000803010FFB9F0E6012096A9F08C3038F404
:10067000839580936100629686ED90E004C01F7BB5
:100680006B9687E593E0C817D90710F06C0177CF18
:100690006E0175CF44CF5DCFEBE295989798C098E7
:1006A0004CC016FD02C0BC3098F5F093610070910B
:1006B0007400715F16FD7093740010643EC01F7D5E
:1006C00001C0106280916200815050F080936200FE
:1006D00016FF0BC0C0E0DFEFAF2EBADEA4E01FC0F4
:1006E000EB3209F4EDE216FD34C07BE193DEBFDEB0
:1006F00073E390DE00FFD0CF14FD89DD68B1612780
:1007000065FDF8CF7ADEA92F6F13AFEFAC3038F468
:1007100074DEC80FD91FA61E7FDEBBE001C0BA2F52
:1007200000FFBFCF14FD73DD68B1612765FD03C015
:10073000AB17AF1FF5CFAA9599F7D0DD16FF97DE5F
:10074000809162008F131E7FBF1208958F918F9149
:10075000E6CEC0E0D0E070E0A72E8091610082304C
:1007600030F47091740080E090E860E03ADE70DE72
:100770007EDEC0E0D8EB7BE0A72E6ADEAFEFCFCF06
:1007800000240FBEEFE5F4E0FEBFEDBF0292E036BD
:10079000F00509F4EEE1E015F005C1F781B78093AB
:1007A0006000A4B6F4BFF8BB81E087BB88E285BBDC
:1007B00088E284BB80E182BB80EB81BB82E083BFA7
:1007C00081E08EBDF5BD88E181BD88E081BDCADCD8
:1007D000E6DCD6DC7894A0FAAF1226F490DC96DC46
:1007E0009CDC71CEA2FE04C098DC89DC00686BCE74
:1007F000A1FE02C099DC67CEF894A3FE05C07FDCA1
:100800007EDC8BDC8ADCFBCFAADC4A2D58E040FF83
:100810007DDC40FD89DCA4DC46955A95C1F7F4CF18
:101C0000E4E0FFE5FEBFEDBF00E0ECEBFEE0C0E886
:101C1000D0E0A0E6B0E042E045BD5CEE539571F047
:101C200040EC04BD48BFA03619F0E8B6E6FC46C05B
:101C30008299F9CF04BD48BFE8B6E6FCE1C1829BBA
:101C4000FBCF04BD48BFE8B6E6FCE8CF8299FBCFE6
:101C500034B404BD48BFE8B6E6FCD2C1829BFBCFDA
:101C600024B4022C030C802C07940694402C069478
:101C70008008809420943094409460EE83E084BC8B
:101C800048BFE8B6E6FCBCC1829BFBCF84BC48BF22
:101C9000E8B6E6FCC3CF8299FBCF0894E8B6E6FC31
:101CA00023C0829BFBCFE8B6E6FCB8CF8299FBCF7E
:101CB0008894E8B6E6FC18C0829BFBCF43BC87E162
:101CC000929A8A9A34BC48BFE8B6E6FEFDCF929855
:101CD00024BC48BFE8B6E6FEFDCF8A9589F7C0E68A
:101CE000D0E060E081E00BC0679548F6815068F570
:101CF0005CEE0994CA17DB07D1F0699188E066951C
:101D0000929A34BC48BFE8B610F0E7FC02BBE6FE8E
:101D1000FACF929808F0929A24BC48BFE8B610F027
:101D2000E7FC02BBE6FEFACF8A9549F7E3CF929A29
:101D300034BC48BFC0E8D0E0A0E6B0E0E8B6E7FEBB
:101D4000FDCF8A9802BB6ACF80E060E898CFECEBC9
:101D5000FEE0C0E8D0E0F8CF009000000090000066
:101D60000090000000900000009000000090000033
:101D70000090000000900000000000006B3121F78F
:101D8000562E3796E1CF962E56263496DDCF762EF8
:101D900056263496D9CF662E56263496D5CF6E3039
:101DA000B1F656263596D0CF69935626CF3584E0C6
:101DB000D80768F681E0681A700A09F43C96C4CF27
:101DC0006511C5CFC0E8D0E0699199918991FD0175
:101DD0007BE170839182028372E073837EE074837F
:101DE0006583068317966130A1F48BE0838388E0D6
:101DF0008D93EF01ECEDFFE185918D93E43EE1F7EA
:101E0000FE01819161918627EA17FB07D9F78D932F
:101E10009ECF6D3151F5792F90E0039683839283A5
:101E200003970D938A95E9F789916991603380074B
:101E300094E0790779F460878991803059F4699149
:101E400060308EE131F0613083E919F0623087E073
:101E500009F482870D93D5CF8017900709F5D990A3
:101E6000C9905601AA0CBB1CCCCF6330E1F06230A4
:101E700041F2603131F2613121F2663069F3623151
:101E8000F1F1833F73E0970758F4643109F166314B
:101E900069F127966531C1F16331F9F10000000065
:101EA00080EC8683AECF90398FE071F0913982E07B
:101EB00059F092398AE041F0943982E329F0903860
:101EC00080E011F0913861F78D9383E0838399CF9F
:101ED00049D0EF01F5018FD076FDFDCF65916D936F
:101EE0000197E1F75F01FE010D938BCF3BD011E02D
:101EF0003ED06DB36D930197D9F70D9382CF47D044
:101F0000000080E092E0689416E06FEF0EF06991B7
:101F10002ED00197D1F7E89474CF8F7F61E07F01D5
:101F2000F5010990199068D032960297D1F70F0108
:101F3000F501500163E0E03C7FE1F70719F058D06C
:101F4000F7015FCF0BD065E009D061E107D0F8CF92
:101F500077B770FDFDCFE199FECF0895F9DF67BF38
:101F6000E8950895039692838383039708953AD062
:101F7000DFBACEBA0894C01ED01E762FE09A6DB399
:101F8000671312FF08957DBBE29A1CBB08957F0181
:101F9000E0E0FEE063E0B0972FD0E9F76F01F701D2
:101FA0000895000000000000000000000000000094
:101FB0000000000000000000000000000000000021
:101FC000687474703A2F2F6769746875622E636F36
:101FD0006D2F73696D2D2F7467792F00415652490B
:101FE00053505F3277B770FDFDCFE199FECF089572
:101FF00003D065E001D061E1F5DF67BFE8950895A2
:00000001FF
